:1051AC0020496E697469616C697A696E6720202088
:1051BC002000202020202020202020202020202003
:1051CC0020200033302E3220202000002040608030
:0351DC00A0C0FF71
:0853BB00C11AC11D41123200AC
:102A4200E92FF9EA3EFAE4121C91901189E0FCA305
:102A5200E0FD90579375F00C121EA5EC75F00CA4D6
:102A62002583F583E493FB740193FA74029322F9AC
:102A720090118BE0FCA3E0F5828C837415121E94F6
:102A8200E92582F9EA3583FA021D7CFFE5F08FF031
:102A9200121DDF901189E0FEA3E0FF90579375F0BD
:102AA2000C22F990118BE0FEA3E0FF7C007D151251
:102AB2001CB3E92FF9EA3EFA229011A07B017A11A8
:102AC200798DEBF0A3EAF0A3E9F022FE855D828521
:102AD2005C83740693F822F0A3EFF0855F82855E33
:102AE2008322F990118BE0FEA3E0F5828E83222FE0
:102AF200F9EA3EFAE4021C91901222E0FCA3E0FD06
:102B0200A3E0FEA3E0222FF9EA3EFAE4021C91E0E0
:102B1200FCA3E0FD7A007B01AE0422900005121CAA
:102B220030FF900006121C30FD900004021C30FDA4
:102B3200E5F08DF0021DDF900003021C30FFEC4E29
:102B4200FEED4FFF22E675F015A4F582E92582F924
:102B5200EA35F0FA121D7CFDE5F022E0131313545E
:102B62000325E0FFE433FE74F92FF974073E22F9DE
:102B720090110CE075F015A4F58285F083121DA763
:102B8200E5F0222FF9EA35F0FAE92402F9E43A22D3
:102B92004EFFEDCF8FF0121DDF855D82855C8322B3
:102BA200F990118BE0FEA3E0FF7C007D15021CB3BF
:102BB200EEF0A3EFF0F5828E83222FF9EA3EFAE4DB
:102BC200021C91FDEF6B7E005401222FF9EA35F0D1
:102BD200FA121C30D322E675F015A4FF22E0FCA302
:102BE200E0FDEC22901116A3E0FAA3E0F5828A83BD
:102BF200227E007F02021BF1F99001F8021C30E0F4
:102C0200FCA3E0FDAE04780722E0FCA3E0FDF58220
:032C12008C83228E
:062A1200E4901232F022F4
:0759FA009012327401F0224B
:10574B00C203C201C200C204C210E4F533C207C2D5
:08575B0008C202C20DC20C22BB
:1052A800122ACE122BD8122A692FF9EA35F0AF014B
:1052B800F55E8F5F8F82F583E5822408F582E435F9
:0F52C80083F583E0FFD3940440059012C2EFF00A
:0152D70022B4
:105179009012A6122BB2A3A3A3122A69F5828A83DD
:105189007F02121EDB9012A6E0FCA3E0F5828C835D
:10519900740693F8E6FFA3A3A3122A69F5828A830A
:0351A900021EDB08
:105212003006247E577F93EFB55D0BEEB55C071227
:1052220051797F0A80137E577F9F1251797F0A122C
:1052320047B17F090249187F091249187F091247AD
:02524200B12297
:10586800E490110EF0C202200605D206125212026E
:0258780052A834
:0F2A2100122ACEA607AF5DAE5C1251790252A801
:10551700300620122ACEEF26F6122ACEE6FFB4185E
:1055270004E4F68006EFB4FF027617122ACEE6FFF0
:04553700122A2122F1
:0A59BB007F0B1249187F0B0247B161
:10587A00122B392408700A7F0F1249187F0F12471A
:02588A00B12249
:104D12001259C512588C75BB06C2EDD2EC30EDFDAE
:104D2200E5BFD3947F4004D2228002C22275BB0722
:104D3200C2EDD2EC30EDFDE5BFD3947F4004D22327
:104D42008002C2233022093023037F24227F2522BE
:084D52003023037F26227F2796
:014D5A002236
:08555F00AB07AF031BEF601A5C
:10556700901270121E630000445C90127074FF1258
:0A5577001E24EC4D4E4F60E280F060
:015581002207
:100C9A00E4F584124D12901233EFF0124BE79012E2
:100CAA0033E0FF12592BE4F58475CFE4F58443F65B
:100CBA0002124A141258AF90126374FFF0A37451CF
:100CCA00F0A374BEF07BFF7A5179AC1251451248F9
:100CDA000F124D5B1254F2125A1A905793122A6647
:100CEA00F9900008121C30D394054007900008E4DC
:100CFA00121C91E4901189F0A3F0E490118BF0A3F7
:100D0A00F0122A95121EA5EE122A5E122A7154FEBC
:100D1A00122B31122A9DEF121EA5EE122A5E122AFA
:100D2A00E4122A7D54FD122A8D121EA5EE122A5EA5
:100D3A00122A7154FB122B31122A9DEF121EA5EEB4
:100D4A00122A5E122AE4122A7D54F7122A8D121EE2
:100D5A00A5EE122A5E122A7154EF122B31122A9D25
:100D6A00EF121EA5EE122A5E122AE4122A7D54DF21
:100D7A00122A8D121EA5EE122A5E122A7154BF1271
:100D8A002B31122A9DEF121EA5EE122A5E122AE4B8
:100D9A00122A7DFFE5F054FEFEEF547FFFEE122A81
:100DAA0090121EA5EE122A5E122A71FDE5F054F980
:100DBA008DF0121DDF122A9DEF121EA5EE122A5E79
:100DCA00122AE4122A7DFFE5F054E7122A90121E35
:100DDA00A5EE122A5E122A71FDE5F0549F8DF012DB
:100DEA001DDF122A9DEF121EA5EE122A5E122AA4F8
:100DFA00122B8BFA121D7C54F8122B31901189E0B8
:100E0A00FCA3E0122A542FF9EA3E122B8AFA121D89
:100E1A007C54074450FFE48FF0121DDF901189E0E3
:100E2A00FEA3E0122A9D121EA5EE122A5E122BA222
:100E3A00900004122A42900005122AF1122A9DED0E
:100E4A00122A5A122BA2900006122A429000071266
:100E5A002B08122A9DED122A5A122AA4900008126F
:100E6A002A48900009122AF1122A9DED122A5A12D2
:100E7A002AA490000A122A4890000B122B08122A60
:100E8A009DED122A5A122AA490000C122A489000A8
:100E9A000D122BBC122A9DED122A5A122AA4900076
:100EAA000E122A4890000F122BBC122A9DED122A0C
:100EBA005A122AA4900010122A482FF9EA3EFA90F0
:100ECA000011E4121C91122A9DED122A5A122AA428
:100EDA00900012E4121C91901189E0FCA3E0122AFE
:100EEA00542FF9EA3EFA9000137463121C91901180
:100EFA008BA3E0FFC007901189E0FEA3E0122A9DB0
:100F0A00121EA5EE122A5EF990118BE0FE7C0012E9
:100F1A002AB1900014D0E0121C9190118CE004F0D8
:100F2A00700690118BE004F090118BE07004A3E03E
:100F3A0064186003020D0B90118AE004F0700690A9
:100F4A001189E004F0901189E07004A3E064026062
:100F5A0003020D04755C57755D93908002E49390CB
:100F6A001234F0D3940940037403F012598FD2AFAC
:100F7A0012588C1256271217117F0412496E7533B4
:060F8A0001E490110EF0DD
:100F90007F407E0D7D037C009007FFE0F8A3E0F921
:100FA000A3E0FAA3E0FBC3121DFE50189007FF1246
:100FB0002AFD2401FFE43EFEE43DFDE43CFC9007F5
:100FC000FF121E57301C07C21C7F0412496E1246C6
:100FD00091EF60097E577F937D011237181246F218
:100FE000EF60097E577F9FE4FD12371830053412F9
:100FF0002AFAFFEF24FFFFEE34FFFEED34FFFDEC95
:1010000034FFFC901222121E57122AFAFFEC4D4EAA
:101010004F7010901233E0FF7BFF7A5179CF124866
:101020006AC205124AB49011A9EFF070030215606C
:10103000E014B41600400302155D90104875F003EB
:10104000A4C58325F0C5837302108A0210BD021166
:10105000600211F30210EB0210CA0210DB02135AF5
:101060000213ED0214290213B802146602120302DD
:10107000126E0210C30212E402133E02134C021558
:101080004302154702154E021555122AFAFFEC4D80
:101090004E4F700302155DC205201A0DE49000004A
:1010A000F0125A20C20F02155DA20BB3920B300B47
:1010B00007C229D20F02155DC20F02155D1259BB7E
:1010C00002155DC202C20602133830000612567DB8
:1010D0000213EA12574BD2000213EA3001051256EE
:1010E0007D800512574BD2010213EA125868300076
:1010F00027122ADDC083C082122B117802CEC313BF
:10110000CE13D8F95401FFED54FB122BC57802C35E
:1011100033CE33CED8F98028300134122ADDC08393
:10112000C082122B117803CEC313CE13D8F9540109
:10113000FFED54F7122BC57803C333CE33CED8F965
:10114000122B3FD082D083EEF0A3EFF00213B23027
:10115000040612567D02155D12574BD20402155D2E
:10116000125868E53370030211EAE55F2402FFE4D8
:10117000355EFAA9077B01C001122ADD122B5DA89A
:1011800001FC7D01D001122BF3122ADDC083C08245
:10119000122BDF1313135403FFEC54E7FCEF24016D
:1011A000FFE433EF540333333354F84CFFEDD08274
:1011B000D083CF122AD9122BDF13131354036403E5
:1011C000700C122ADDEC54E7AF05F0A3EFF0122A01
:1011D000DD122B5DFA7B01E55F2402FFE4355EA89A
:1011E00007FC7D01122BF30213B212574B7533012A
:1011F00002155D30100512567D800512574BD21036
:101200000213EA12586830075D122ADDC083C082DB
:10121000122C01CEC313CE13D8F95403FFEC54FEA5
:10122000FCED547FFDEF2401FF7E00EF54037807AF
:10123000C333CE33CED8F9122B3FD082D083EE12F7
:101240002AD9122C01CEC313CE13D8F95403640348
:10125000700F122ADDEC54FEFFED547FCFF0A3EFA8
:10126000F0125336800312574BD20702155D300837
:101270006B12567D90111BE014601C1460191460F1
:101280002914602614603A2405704C122ADDC083AC
:10129000C082E054F98034122ADDC083C082E05459
:1012A000F9FEA3E0FFEE44028011122ADDC083C0E4
:1012B00082E054F9FEA3E0FFEE4404D082D08380A4
:1012C00012122ADDC083C082E04406FFA3E0D08270
:1012D000D083CFF0A3EFF0125336800312574BD2D6
:1012E000080213EA3006187E577F93EFB55D0CEEC7
:1012F000B55C08755C57755D9F80048E5C8F5D12D0
:101300002ACE122BD8122A66900008122BCD9404F4
:101310004007900008E4121C91122ACE122BD8121A
:101320002A66900009122BCD94044007900009E42E
:10133000121C91C20212586812521202155D755C9D
:1013400057755D9312574BD2030213EA755C5775BC
:101350005D9F12574BD203021460125868122ADDA7
:10136000C083C082E0FEA3E0FF5401FBEF54FEFF08
:10137000EB6401FD5401FBEF4BFFD082D083EEF014
:10138000A3EFF0ED702C122ADDC083C082122BDF98
:10139000C313ED135401FFED54FDFDEF640154013F
:1013A00025E0FFE433FE122B40D082D083EEF0A381
:1013B000EFF012533602155D30062F122ADDC0837E
:1013C000C082122B117806CEC313CE13D8F9540164
:1013D000FFED54BF122BC57806C333CE33CED8F9F8
:1013E000122B3FD082D083121708021460300637C8
:1013F000122ADDC083C082122BDFC4F854F0C8ED7E
:10140000C4540F485401FFED54EFFDEF6401540143
:10141000C4F8540FC868FFE4C454F048FE122B40CF
:10142000D082D0831217088037300634122ADDC0EC
:1014300083C082122B117805CEC313CE13D8F95472
:1014400001FFED54DF122BC57805C333CE33CED860
:10145000F9122B3FD082D083EEF0A3EFF012533677
:1014600012586802155D20060302155D2002030272
:10147000151990110EE0600302150B122ACEE6FE3C
:1014800090110CE0FF6E607B90110BE0FDEEB50556
:1014900008C202122A2102155D122B9B122A661223
:1014A0002B715418122ACD122B4754E7122B92128B
:1014B0002A66122B715460122ACD122B47549F12A8
:1014C0002B92122A66F990110CE075F015A4FFE931
:1014D000122B85FAC003C002C001122ACE122BD8EB
:1014E000122A66122B85A801FCAD03D001D002D0D0
:1014F00003122BF3122ACEE690110BF07F0412494F
:101500006E805A90110E7401F0805290110EE0041A
:10151000F064047048C2028044D202C21BC21EE5BD
:1015200033700330100DE490110EF090110B74FF26
:10153000F0800690110E7401F0122ACEE690110C84
:10154000F0801A7F0180027FFF125517800F122B47
:10155000E67F018005122BE67FFF121EDB121711BA
:10156000301D0E901232E07006A3E0FF125719C230
:101570001D7B017A11798D125363EF7003020F9076
:1015800090118FE0121EB115E60416070515B6146A
:1015900015A61615AC1715BB1A15CF1B15DA1D1598
:1015A000E01E00001631D20BD20F8004C20BC20F16
:1015B0001233D9021631D21A02163190119D122A15
:1015C000BE121C17FE901233E0FF6E70648005900F
:1015D0001233E0FF1257C20216311259FA021631C5
:1015E000122A12021631122ABB122B39FF90123323
:1015F000E06F703D300B329011A004122AC5122BFF
:101600001DFB1242218022122ABB122B39FF90129D
:1016100033E06F701C300B119011A004122AC51218
:101620002B1DFB123F651254F2901233E0FF12574C
:1016300032200B0302157190118FE014603B14608F
:101640002324FB60541470030216D324F9600302B0
:1016500015717B017A11798D9011A6122AC4125846
:101660007A0215711216F490119D122AC4122B39A8
:10167000900000F0125A2080541216F490119D121E
:101680002AC4122B39900000F01254F212360A12BA
:1016900033D97F0512496E80341216FE9011A312C1
:1016A0002AC4122B39FF122B2BFD900005121C307F
:1016B000FBC0039011A3E0FBA3E0FAA3E0F99000C4
:1016C00006121C309011B9F0D003123EC112599A83
:1016D0000215711216FE9011A3122AC4122B39FFA3
:1016E000122B2BFD900005121C30FB12303E1259BC
:0416F0009A021571D4
:1016F40012589E7B017A11798D2212589E7B017AB1
:1017040011798D22EEF0A3EFF01253362212360A2D
:041714001233D92291
:0F4BE70075FFDE75FFAD75840F759601758C2017
:104BF600E49012A8F0A3F09012A9E004F0700690D9
:104C060012A8E004F09012A8E0B44EEBA3E0B420A2
:014C1600E6B7
:104C1700759701758A8843B730E4F5841257631294
:0B4C270056981245C71259C5025A01E9
:1057630075840F75A41175A57CE4F5A675A7E0757E
:08577300E12575E344F58422F1
:075A0100E4F58475D4842252
:10569800E4F58443E60875DA3175DB3175DC31757C
:0A56A800DD3175D983D2DEF58422CE
:0A59C50075E8C175BCF875D1032226
:10588C00751912751A35E4F513F5BB75E8D143E7B4
:02589C000222E6
:032A3000024EBC97
:104EBC00C0E0C083C082C0D075D000C006C2ED0572
:104ECC001AE51AAE197002051914F5828E83E5BF26
:104EDC00F00513E513B40409751912751A35751319
:104EEC00008513BB75E8D1D006D0D0D082D083D04A
:024EFC00E032A2
:105483007F07124918901238E0FF1249189012371B
:10549300E0FF124918901236E0FF124918901235B6
:0554A300E0FF024918C2
:1054A8007F071247B1901238E0FF1247B1901237C8
:1054B800E0FF1247B1901236E0FF1247B190123563
:0554C800E0FF0247B106
:104C32009012AA122BB2122A66122BFAD3940540B2
:104C4200079001F8E4121C919012AA122AE8A3A379
:104C5200A3122A69F5828A837F01121EDB9012AAAF
:104C6200122C0B122A66122BFAFF8D828C83A3A3BD
:0B4C7200A3122A69F5828A83021EDB70
:10371800901268EDF0901266122BB2740793F8E6D7
:1037280024FD606724FD606B24FA607314607314D1
:103738006073240E60030237F9901266E0FEA3E07E
:10374800FFF5828E83740893FC740993F5828C8349
:05375800E024F87030D0
:10375D008F828E83122A66122BFA901269F0E00482
:10376D00F0B40502E4F0901269E0FD901266E0FEFF
:10377D00A3E0FF9001F8ED121C91124C321253365A
:10378D0012360A0233D91252127F0402496E901278
:10379D0068E060030254830254A802360A025336CD
:1037AD00E4901269F0901266122C0B740A93FE7459
:1037BD000B93F5828E83E075F015A4FF8D828C83BB
:1037CD00122A662FF9EA35F0FAE9240AF9E43AFAF1
:1037DD00901269E07E0029F9EE3AFA121C17901248
:0C37ED006AF0901269E004F0E0B404B946
:0137F90022AD
:0B598F00901234E09051D793F5D32222
:1053C30042110100004210AC00004210A70000C1CE
:0553D30021C120C11FF3
:104A65009010A7E475F001121D50FCE5F064404C70
:104A750022D3901102E09400901101E064809480AB
:104A850022E0FEA3E024AEF582741022E0FBA3E051
:104A9500FAA3E0F98E82758300229010A7F0A3F0A7
:0F4AA500229010A3E004F0229010A2E004F0226F
:0A59CF00C220C221E49010ABF022C8
:1055E800E4901101F0A3F09010ACF0A3F0A3F01236
:1055F8004A9F9010A2F0A37440F0E49010AAF02201
:065A08001259CF0255E81F
:10570000E4F5848FC343C30175C04475CF8EC2C313
:0957100043E6029010A904F02206
:10589E00E4F58420C7FDC2C2125A08E49010A9F0A4
:0158AE0022D7
:0B599A00E4F584D2C29010A904F022B2
:0D592B00AE071257009010A6EFF0025A08C8
:1054CD00E49012ACF0A3F0302002FF222021FDD297
:1054DD00209010A4E4F0A37410F09010EFEFF0E41E
:0454ED00A3F07F01A8
:0154F1002298
:1051110030200A9010A4E07002A3E070037F002207
:105121009010A5E024FFF09010A4E034FFF090105F
:10513100F0E0FE04F074F12EF582E43410F583EF13
:04514100F07F0122D8
:0B59A500302007C220D2211258F1224E
:0E58F100AF84E4F58420C7FDC2C4D2C58F8405
:0158FF002286
:1044EE0090123AEBF0A3EAF0A3E9F09010A9E07075
:1044FE0002FF2290123DE0FE6005D3941040037F30
:08450E0000221254CDEF6044BD
:10451600E490123FF090123DE0FF90123FE0FEC3A0
:104526009F501A90123A124A91121C30FF125111E2
:10453600EF7002FF2290123FE004F080D8E4901062
:10454600ABF01259A590123EE070032021FD9010A9
:04455600ABE0FF22B5
:03455A007FFF22BE
:0E3E1A00901274EBF0A3EAF0A3E9F0A3EDF030
:103E2800E4FF124A7650012253E6FD9010A7124A89
:103E3800863EF583E0FF124A657003124A9F124AD4
:103E4800A67003124AADE4FE901277E0FDEEC39D22
:103E5800502FEEC39F502A9010A7E0FC124A883CCE
:103E6800F583E0FD901274124A91ED121C91124AEA
:103E7800657003124A9F124AA67003124AAD0E805B
:103E8800C7EEC39F5013124A657003124A9F124A25
:103E9800A67003124AAD0E80E8901102E024FFF0EC
:103EA800901101E034FFF043E602901277E0FEEF54
:083EB800C39E50028002AF0618
:013EC00022DF
:0C2A3300124A7640047F0180027F0022DE
:032A1800022DA1EB
:102DA100C0E0C0F0C083C082C0D075D000C000C0F8
:032DB10006C00752
:102DB400C226AFC1EF121EB12DEA082DEA102DFA7A
:102DC400182DFF202E0C282E39302E44382E4C601E
:102DD4002E47682E4C702E47782E54802E54902EF9
:102DE400C4A000002ED29010EFE0F5C2C2C590102E
:102DF400EEE4F0022ED49010F080289010AB74FD15
:102E0400F0D2C4D2C5022ED49010F0E0FF9010EEA0
:102E1400E0C39F5014E0FF04F074F12FF582E43412
:102E240010F583E0F5C2022ED4D2C49010ABE4F0C6
:102E3400C221022ED4D2C59010AB74FEF0022ED45F
:102E4400022EC9D21F022ED49010A1E4F0022ED477
:102E54009010A1E07020E5C2F0E0FFC39010A3E061
:102E64009F7480F89010A2E064809850031255E893
:102E74009010A1E004F09010A3E024FFF09010A2C1
:102E8400E034FFF09010AC124A863EF583E5C2F0C0
:102E94009010ACE475F001121D50FEE5F064404E54
:102EA40070069010ACF0A3F09010A1E014F0702024
:102EB400901102E004F07018901101E004F0801009
:102EC400301F0DC21F9010EEE4F0D2C58002D2264E
:102ED40030260EC2C6D2C6C2C5C2C4D2C2C226C21F
:032EE40021C2C345
:102EE700D007D006D000D0D0D082D083D0F0D0E0A9
:012EF70032A8
:055A0E00A2C7E433FF14
:015A13002270
:1049C200EFF0A3ECF0A3EDF0A3EBF0A3EAF0A3E980
:1049D200F0227403F0A374E8F0A3E584F0E4F58414
:1049E20022D2C4D2C5D2C2C2C3E49012C4F0FF2202
:1049F200E0FBA3E475F001121D66A9F0FA22E0259E
:104A0200E044A0F5C27F032274FFF5F0121D504569
:024A1200F02290
:065A1400C2C253E6FD22B0
:0634FA009011AA1249C264
:103500009011B31249D420C7FDC2C4D2C2D2C5E4BF
:10351000FF9012C4F030C3FDAEC1EE24F860232446
:10352000F8601F24F8602924F8603024F8603424FF
:10353000F870030235BD24F870030235C524380243
:1035400035CDEF70069011AA124A00C2C50235D3DC
:103550009011ABE0F5C27F050235D39012C474031D
:10356000F08070EFB4050B9011ABA3E0F5C27F06BD
:103570008061EF640670349011B2E09011AD700577
:103580001249F28008E0FBA3E0FAA3E0F9121C174D
:10359000F5C29011B1E024FFF09011B0E034FFF0DB
:1035A000E07002A3E0702C7F078028EFB40706D2FA
:1035B000C47F09801E9012C47405F080169012C456
:1035C0007404F0800E9012C47406F080069012C449
:1035D0007401F0EFB40904C2C380259012C4E0B4B2
:1035E000030B9011B3124A0A60031249E39012C40C
:1035F000E06008C2C5D2C4C2C38005C2C30235158B
:0936000020C7FD9011B5E0F5842E
:01360900229E
:0632AF009011C21249C299
:1032B5009011CA1249D420C7FDD2C2C2C4D2C5E4F6
:1032C500FF9012C4F030C3FDAEC1EE121EB132F84C
:1032D5000032FB0832FB10332018332B2033332800
:1032E500334E30335638335E40336E503396580084
:1032F5000032F802339CC2C5EF70099011C2124A20
:10330500000233A2EF640160030233A29011C2E010
:1033150025E044A1F5C27F040233A29011C3E0F574
:10332500C27F050233A29012C47403F0806FEFB41C
:10333500050B9011C3A3E0F5C27F068060EFB406CC
:1033450006D2C57F01805680189012C47404F0809F
:103355004C9012C47406F08044EFB404047F0280DC
:103365003C9012C47405F080349011C51249F2E501
:10337500C2121C7F9011C9E024FFF09011C8E034FF
:10338500FFF0E07002A3E07004C2C280107F0280EB
:103395000CD2C47F0980069012C47401F0EFB40901
:1033A50004C2C380259012C4E0B4030B9011CA1265
:1033B5004A0A60031249E39012C4E06008C2C5D20C
:1033C500C4C2C38005C2C30232CA20C7FD9011CC56
:0333D500E0F5849C
:0133D80022D2
:10317D009011F7EFF09011FA1249CB9011F8ECF095
:03318D00A3EDF0BF
:10319000755600543FF557543F6058C374409557D7
:1031A000FFE49556FE9011FDE0FCA3E0FDC39FEC0B
:1031B0009E50068C548D5580048E548F551232814A
:1031C00060037F02229011F9E02555F09011F8E09C
:1031D0003554F09011FFE0700B9011FBE5548555CC
:1031E000F0121D50C39011FEE09555F09011FDE0D6
:1031F0009554F09011FDE0F554A3E0F555D3E55555
:103200009400E55494004076E5559440E5549400CC
:10321000500F12328160037F0222E4F554F555808D
:10322000DC9011F7E0FFA3E0FCA3E0FDA3E0FBA32B
:10323000E0FAA3E0F99011B0E4F0A37440F090112B
:10324000FFE09011B2F01234FA9012C4E060037FF4
:10325000022274C02555F55574FF3554F55490116C
:10326000F9E02440F09011F8E03400F09011FFE014
:10327000708B9011FB75F040121D500231FD7F00E4
:10328000229011F7E0FFA3E0FCA3E0FDA3E0FBA385
:10329000E0FAA3E0F99011B0E554F0A3E555F09001
:0F32A00011FFE09011B2F01234FA9012C4E02244
:1057AB009011C8E4F0A304F01232AF9012C4E06081
:0757BB00037F01227F0022A1
:1056B2009012C3EBF07B017A1279C39011FDE4F0F2
:0A56C200A304F0E4A3F012317D22EE
:10558200C007901218E0FFA3E09011C8CFF0A3EF7C
:10559200F0D0071232AF9012C4E060037F01227F85
:0255A2000022E5
:1056CC00C007901220E0FFA3E09011FDCFF0A3EFF4
:0A56DC00F0E4A3F0D00712317D22A4
:1056E6007B01E4901252F0227422F0A3EFF0A32281
:0A56F6007B01E4901252F07D0422C3
:0E4E770090124EEBF0A3EAF0A3E9F0A3EDF0E9
:104E8500E4901253F090124EE0FBA3E0FAA3E0F990
:104E9500A3E090123DF0901252E090123EF0E4FF34
:104EA5001244EEEFB4FF0D901253E0FE04F0EEC392
:064EB500940340D17E00D1
:014EBB0022D4
:0B536300901294EBF0A3EAF0A3E9F035
:10536E007E007F007D10121EDD901294E0FBA3E004
:10537E00FAA3E0F97D10123E1AEF7002FF227F01B0
:01538E0022FC
:10486A009011E31256EE7413F0121C179011E6F031
:10487A00900001121C309011E7F0900002121C30D7
:10488A009011E8F0900003121C309011E9F09000AA
:10489A0004121C309011EAF0900005121C3090119D
:1048AA00EBF0900006121C309011ECF07A1179E3CB
:0848BA001256E67D0A024E775A
:105719009012781256EE7403F0A374FFF07A12799E
:09572900781256E67D04024E7769
:1057C20090127C1256EE741CF0A374FFF07A1279D8
:0757D2007C1256F6024E772F
:10573200E4901280F0A3EFF0A3740AF0A3EFF07AE2
:095742001279801256F6024E772E
:10560800E0FEA3E0A60608F6E4F584C2AF43B701BE
:0F56180022E475F001021D66EEF0A3EFF0A3226D
:10506D00AB84A2AF9227E4FCFDED901284121E5783
:10507D009012867864125608438F02438F0118E60A
:10508D00FE08E6F5828E83E4F053B7FEF58FA22776
:06509D0092AFAF038F8407
:0150A30022EA
:024EFE00AB0502
:104F0000AA84A2AF9228E4FCFDED901288121E57ED
:104F1000EBFF3395E0FEEFF44E601C90128A78664A
:104F2000125608758F0118E6FC08E6F5828C83EBB3
:0F4F3000F053B7FEE4F58FA22892AFAF028F8443
:014F3F00224F
:10475300901254125620ECF0A3EDF0A3EAF0A3EB71
:10476300F0901258E07002A3E06042901254E0FE11
:10477300A3E0FFA3E0FCA3E0F5828C83E0FD124EEF
:10478300FE901259E024FFF0901258E034FFF090AD
:104793001257E004F07006901256E004F0901255A0
:0E47A300E004F070BC901254E004F080B422E8
:0859E200E4900C9FF0A3F022F9
:10545D00900C9FE0FEA3E0FF12506D900C9FE0FEBC
:10546D00A3E0FF7C0C7DA17B007A04124753E490EE
:06547D000C9FF0A3F022D9
:0A41A000A90590125AEEF0A3EFF00B
:1041AA00EE54FCFE900C9FE0FCA3E0FD7002EE6C66
:1041BA00604CED4C600312545D90125AE0FEEE54CE
:1041CA00FCFE7F00900C9FF0A3EFF090125C125659
:1041DA0020740CF0A374A1F07E0490125C1256199C
:1041EA0085F082F583E493FD90125E12561985F0EC
:1041FA0082F583EDF0EF1F70011EEF4E70DC901216
:10420A005AE0FCA3E0FDEC5403FC74A12DF5827482
:06421A000C3CF583E9F005
:01422000227B
:104FBE00901240125620EBF0A3EAF0A3E9F0901203
:104FCE004574FFF5F0121D6645F0601E90124012FA
:104FDE005619AFF0FE901242E0FBA3125619A9F03B
:0B4FEE00FA121C17FD1241A080D42213
:1058D1000001FF00FF000001010000FF00FF0100C7
:0D53D800C10BC10F44122200000000C105EE
:10447E0090128CA3A3E0FEEE2290128CA3A3A3E0D5
:10448E0022EF4D24D1F582EE3458F583E493FF905C
:10449E00128DF0A3E52BF0EF252BF52BE0652B22EB
:1044AE00FFE4FEFDFCEF22855F82855E83E0FEA3C6
:1044BE00E022901297E0FBA3E0FAA3E022AFB0FE59
:1044CE00EF5403FFE47810021E0FEF4BFFEE4AFE8F
:1044DE00ED49FDEC482290128CA3E0FDE4FEED22A6
:104A1400D295C2961255A4E4FCFDC004C005C0069C
:104A2400C0071244CBD003D002D001D0001244D826
:104A34008F378E368D35F5348F3D8E3C8D3BF53A70
:104A4400AF807538008F39AF90753E008F3F7B0083
:104A54007A0079408B2F8A3089318B2C8A2D892ECC
:014A6400222F
:10462F00E52E2401F9E4352DFA901297E52CF0A32D
:10463F00EAF0A3E9F01244C0F9900054EB7008E9D6
:10464F0065827003EA6583700C901297F0A3740073
:10465F00F0A37440F01244C0F9E52F853083853103
:10466F00826B7008E965827003EA65836013AB2C77
:10467F00AA2DA92EEF121C7F1244C08B2C8A2DF568
:01468F002EFC
:014690002207
:104AB40053E6F7E52F853083853182652C700AE54E
:104AC4002E65827004E52D65837003FF802CAB2F67
:104AD4000531E531AA307002053014F9121C17FFB4
:104AE400900054EB700AE53165827004E53065830B
:0D4AF4007008F52F75300075314043E6085D
:014B01002291
:10577B007E80E4FDEF5E24FF9292C293EEC313FE94
:07578B00D2930DEDB408ED0F
:0157920022F4
:1055A400D296E4FBC295ED25E0FDEC33FC30970484
:1055B400ED4401FDD2950BEBB410E9C296AF05AEF4
:0155C40004E2
:0155C50022C3
:032A1E0002228E03
:10228E00C0E0C0F0C083C082C0D075D000C000C016
:10229E0001C002C003C004C005C006C00720DF0392
:0322AE00022535D1
:1022B100E5126005D51202D21C1255A4E4FCFDC042
:1022C10004C005C006C0071244CBD003D002D00120
:1022D100D0001244D88F2A8E298D28F527AF3DAE24
:1022E1003CAD3BAC3AAB2AAA29A928F8C3121DFE82
:1022F100603DE52A653DFFE529653CFEE528653B36
:10230100FDE527653AFC90128C121E5790128CE065
:10231100FCA3E0FDA3E0FEA3E0FFEC4D4E4F600304
:10232100753203852A3D85293C85283B85273AE579
:102331003270030225331532E5326003022533E59D
:102341002A5401FFE4FEFDFCFBFAF9F8C3121DFE5D
:10235100700C901222121E630000157CD205E53725
:10236100652AFFE5366529FEE5356528FDE5346515
:1023710027FC90128C121E5712448754011244AE4E
:10238100600DE52A5401FFEF60057F0112462F120F
:10239100448754021244AE600DE52A5402FFEF60F7
:1023A100057F0212462F12448754041244AE600D79
:1023B100E52A5404FFEF60057F0312462F1244877C
:1023C10054081244AE600DE52A5408FFEF60057F02
:1023D1000412462F12448754101244AE600DE52AB0
:1023E1005410FFEF60057F0512462F1244875420D9
:1023F1001244AE600DE52A5420FFEF60057F0612FE
:10240100462F12448754401244AE600DE52A5440D1
:10241100FFEF60057F0712462F1244875480124454
:10242100AE600DE52A5480FFEF60057F0812462F4C
:1024310012447E5401FEE4FDFCEE600DE5295401D9
:10244100FEEE60057F0912462F12447E5402FEE41F
:10245100FDFCEE600DE5295402FEEE60057F0A12D7
:10246100462F12447E5404FEE4FDFCEE600DE52986
:102471005404FEEE60057F0B12462F12447E540871
:10248100FEE4FDFCEE600DE5295408FEEE60057FDB
:102491000C12462F12447E5410FEE4FDFCEE600D3A
:1024A100E5295410FEEE60057F0D12462F12447E81
:1024B1005420FEE4FDFCEE600DE5295420FEEE60A3
:1024C100057F0E12462F12447E5440FEE4FDFCEEC1
:1024D100600DE5295440FEEE60057F0F12462F1274
:1024E100447E5480FEE4FDFCEE600DE5295480FE3F
:1024F100EE60057F1012462F1244E45401FDE4FC06
:10250100ED600CE5285401FD60057F1112462F1284
:1025110044E45402FDE4FCED600CE5285402FD6046
:10252100057F1212462F852A37852936852835855C
:042531002734C2DFAA
:0625350020D80330D94C50
:10253B0090128CE580F0C2D9C2D8E0FFFDE5396D71
:10254B0054C06038EFC413135403FDE538C4F8547A
:10255B00F0C8E539C4540F487E00540CFF12448F69
:10256B0030E11090128DE0B401047F1480027F13D0
:0C257B0012462F90128CE0753800F539E4
:0625870020DA0330DB49FD
:10258D0090128CE590F0C2DBC2DAE0FDFFE53F6F03
:10259D0054036035E53FAE3E7802C333CE33CED81B
:1025AD00F97E00540CFFED5403FD12448F30E11001
:1025BD0090128DE0B401047F1580027F1612462F14
:0925CD0090128CE0753E00F53F10
:1025D600D007D006D005D004D003D002D001D00059
:0B25E600D0D0D082D083D0F0D0E03203
:1033D900E4FD3006353002057440FD800E300804E6
:1033E900ED4410FD300704ED4420FD30031C7493B7
:1033F900B55D097457B55C04ED4480FD749FB55DF6
:10340900097457B55C04ED4408FDEDF4FF12577BD0
:10341900E4FD300664749FB55D067457B55C010D13
:103429001244B5FF30E004ED4402FDEEC313EF137F
:1034390030E004ED4404FD1244B57806CEC313CE42
:1034490013D8F930E004ED4410FD855F82855E8371
:10345900E0FAA3E0FBAE027805CEC313CE13D8F988
:1034690030E004ED4420FDEAC4F854F0C8EBC4543C
:103479000F4830E004ED4440FD300F04ED4480FD79
:10348900EDF4FF12577BE4FD30065C200245E5337D
:1034990060010D301004ED4402FD20042430000FBA
:1034A9001244B57802CEC313CE13D8F920E01230F6
:1034B90001131244B57803CEC313CE13D8F930E003
:1034C90004ED4404FD300004ED4408FD300104ED31
:1034D9004410FD7493B55D097457B55C04ED44401F
:1034E900FDED4480FD8004ED4420FDEDF4FF02571D
:0134F9007B57
:1042A20001011226010000000000000000000000D1
:1042B20000000000000000000000000000000000FC
:1042C20000000000000000000000000000000000EC
:1042D20001000017040101FB010112280000000087
:1042E2000101122701000000000000000000000090
:1042F20000000000000000000000000000000000BC
:1043020000000000000000000000000000000000AB
:1043120001000018040103F9010112290000000044
:0D593800F583E493FB740193FA740293224B
:065A1A00E4F50FF50E2279
:104691001253E6EF6058E50E6021150EE509450A53
:1046A10045086043125244AB08050AE50AAA09709D
:1046B10002050914F9EF121C7F802C1252448F104D
:1046C100EF25E025E024A2F582E43442F583E4936A
:1046D100F50EEF25E025E024A3F582E434421259DA
:1046E100388B088A09F50AE50E70037F01227F00E5
:0146F10022A6
:1046F20012538FEF6058E50F6021150FE50C450D41
:10470200450B6043125276AB0B050DE50DAA0C70FA
:1047120002050C14F9EF121C7F802C1252768F11B5
:10472200EF25E025E024E2F582E43442F583E493C8
:10473200F50FEF25E025E024E3F582E43442125937
:10474200388B0B8A0CF50DE50F70037F01227F0079
:014752002244
:102EF800000102040810000003041800000000008C
:102F08001F0000000000180403000000001008045F
:102F180002010000040A0A11110000010102021C4A
:102F280000001C0202010100001010080807000040
:102F3800070808101000008040C020A060E0109032
:102F480050D030B070F0088848C828A868E81898A9
:102F580058D838B878F8048444C424A464E4149491
:102F680054D434B474F40C8C4CCC2CAC6CEC1C9C49
:102F78005CDC3CBC7CFC028242C222A262E212926D
:102F880052D232B272F20A8A4ACA2AAA6AEA1A9A49
:102F98005ADA3ABA7AFA068646C626A666E6169631
:102FA80056D636B676F60E8E4ECE2EAE6EEE1E9EE9
:102FB8005EDE3EBE7EFE018141C121A161E111912B
:102FC80051D131B171F1098949C929A969E9199919
:102FD80059D939B979F9058545C525A565E5159501
:102FE80055D535B575F50D8D4DCD2DAD6DED1D9DB9
:102FF8005DDD3DBD7DFD038343C323A363E31393DD
:1030080053D333B373F30B8B4BCB2BAB6BEB1B9BB8
:103018005BDB3BBB7BFB078747C727A767E71797A0
:1030280057D737B777F70F8F4FCF2FAF6FEF1F9F58
:063038005FDF3FBF7FFFD8
:0959D900E0FBA3E0FAA3E0F922CF
:1058AF007F381258197F061258197D0EE4FF0259DE
:0158BF005F89
:105819009012C5EFF01257D9EF20E7F99012C5E0C1
:04582900FF0250A486
:1057D90075A0FFC2B6D2B5D2B77F14DFFEAFA0EF76
:0557E900902F3E93FF2C
:0157EE002298
:055A2C007F0102581982
:1050A400EF902F3E93F5A07FFF7E00EF1F70011E4F
:1050B400EF4E70F7C2B6C2B5D2B77E007FFFEF1FC6
:1050C40070011EEF4E70F7C2B77E007FFFEF1F70B6
:0650D400011EEF4E70F713
:0150DA0022B3
:1050DB00EF3395E0FE743E2FF582742F3EF583E49B
:1050EB0093F5A0C2B5D2B7D2B67FFF7E00EF1F708B
:1050FB00011EEF4E70F7C2B77E007FFFEF1F7001EE
:05510B001EEF4E70F7DD
:01511000227C
:0C595F009012C6E05FF04DFFF0025819F6
:0E590F00AE071257D9EF20E7F9AF060250DBC2
:1053080090129AEBF0A3EAF0A3E9F090129A1259DE
:10531800D9121C17601790129AA3E475F001121D98
:0E53280066A9F0FA121C17FF12590F80DE2240
:10514500901260EBF0A3EAF0A3E9F0125A2CE4FD0B
:10515500FF12596B9012601259D9125308E4FD7F62
:105165000112596B9012631259D91253087D117FA0
:045175000102596B6F
:0C596B00EF75F040A42D2480FF025819B5
:103B38009011D4E0FF75F0FCA42403F582E5F0347D
:103B480080F583EF75F003A42583AF8222F5832FD8
:103B5800F58375F015EE021EA5FE7A0079017B014A
:103B68009012457403F0A374FCF022E0FBA3E47503
:103B7800F001021D66AFF0FEE0FCA3E0F5828C8345
:103B8800E493FD229011D0F0A3EFF0E49011D6F069
:103B9800A3F022E4F075F0FEEFA4227E007C037D02
:103BA800FC121CB374032FF974803EFA2275F0FCE2
:103BB800EEA42403F582E5F03480F583EE22EFF0DD
:103BC800A3EDF0A3EBF0A2AFE433A3F0C2AF22FD64
:103BD800EDFFEEF0A3EFF022A3F0A37401F0A3220F
:0E3BE8009011D7E004F0229011D6E004F022F4
:10533600301A27202926300B237F407E0D7D037CE3
:10534600009007FFE0F8A3E0F9A3E0FAA3E0FBC3AF
:0D535600121DFE7002D21DD22922D20F229C
:0552D8009012AEEFF0A2
:1052DD001259E2E49012AFF09012AEE0FFA3E0FE9F
:1052ED00C39F5014123BB5123B4C123B61124FBE83
:0B52FD009012AFE004F080E002545D6E
:103A7A007E037FFC7D007B017A007901121EDDE462
:103A8A00FFE4FEE4FD75F0FEEFA4240FF582E5F0F5
:103A9A003400123B55E5822DF582E43583F58374B3
:103AAA000AF00DEDB404DE75F0FEEFA42403F582EE
:103ABA00E5F03400123B55C083C082A3E05407FDF1
:103ACA00ED4420FDD082D0837403F0A3ED123B9C19
:103ADA002414F582E5F03400123B557463123B9CC2
:103AEA002409F582E5F03400123B55123B9B240A67
:103AFA00F582E5F03400123B55123B9B24F9F5821E
:103B0A00E5F03401F5832FF583123B9B24FAF58205
:103B1A00E5F03401F5832FF583E4F00EEE641860C6
:0D3B2A0003023A8D0FEF64026003023A8B34
:013B3700226B
:1048C2009012B07403F0E4A3F01259E27E807F00EC
:1048D2007A1279B012490A7E807F017A1279B11276
:1048E200490A9012347404F07E807F027B017A12AE
:1048F2007934901245E4F0A304F0124FBE12545DD5
:08490200123A7A7F1E0252D81E
:0E490A007B01901245E4F0A304F0124FBE2290
:104D5B00908001E493F46009908000E49364036015
:104D6B00031248C27E007F067D007B017A0779F92A
:104D7B00121EDDE4900000F09007FBE054F8FE7487
:104D8B003BFF9007FBEEF0A3EFF0EE54074470905F
:074D9B0007FBF0A3EFF0227B
:1054F2009012C774FAF0900000E0FFC3941E50149B
:10550200123BA37BFF78017C007D017E037FFC12AE
:045512001BF1C2299E
:015516002272
:10564500900000E0C3941E50121259E2900000121F
:0C5655003B3B123B61124FBE12545D2221
:065A2000125645C22922C6
:04496E00901200EFB4
:10497200123BE17400F07401123BE07401F074FF29
:10498200123BE074FEF0124918901200E0802A9067
:10499200120774FFF5F0121D6645F06022901201B5
:1049A200123B73A9F0FA121C17FF12491890120455
:0F49B200123B73A9F0FA121C17FF1247B180D005
:0149C10022D3
:083EC1009011B7EDF0A3EBF046
:103EC900A3E004F09011BCEFF0A3EBF09011B7E080
:103ED900FF9011BCE0FED39F506B123BB5123B4CD7
:103EE9009011BEF0A3EFF09011BD123B3B9011C0B1
:103EF900F0A3EFF0E49011BAF0A3F09011C0123BD7
:103F0900769011BE123B7D1241A09011BFE004F0E2
:103F190070069011BEE004F09011BBE004F0700649
:103F29009011BAE004F0C39011BBE094FC9011BA6F
:103F3900E0940340C612545D9011BCE004F0A3E084
:103F490004F0023ED5900000E0FF9011B8E0D39F45
:0B3F59005009A3E0C39F40031254F284
:013F6400223A
:0F303E009011CEEDF09011CDEFF09011CFEBF09F
:10304D009011D4EFF0A3EBF09011CEE0FF9011D4DE
:10305D00E0D39F4003023138A3123B3B123B8C90CF
:10306D0011D6E0FEA3E0FFC394FCEE9403502A902A
:10307D0011D0123B8074FD2FF58274033EF583ED64
:10308D00F09011D1E004F070069011D0E004F01230
:10309D003BE870CB123BEF80C6123B389011D2F05B
:1030AD00A3EFF09011D5123B3B123B8C9011D01237
:1030BD003B769011D2123B7D1241A09011D3E004CA
:1030CD00F070069011D2E004F0123BE87003123B51
:1030DD00EFC39011D7E094FC9011D6E0940340CC4F
:1030ED00123B389011D2123B8F9011D6E0FCA3E029
:1030FD00FDC394FCEC940350229011D2123B76AF99
:10310D00F0FE74FD2DF58274033CF583E0FD124154
:10311D00A0123BE870D3123BEF80CE12545D90119C
:10312D00D4E004F0A3E004F0023055900000E0FF7D
:10313D009011CFE0FED39F50209011CDE0FDA3E084
:10314D00C39DFDE49400FCEE7A002DFDEA3CFCC32A
:10315D00ED9F7480F86C985013900000E0FF901173
:0F316D00CDE0D39F5009A3E0C39F40031254F25B
:01317C002230
:033F65009011EDCB
:103F6800123BC6125A149011EEE0FE9011EDE0904B
:103F780011F5123BD7E49011F1F09011EFE0FF90AA
:103F880011F5E0FCA3E0FD7B017A0379FD9012189E
:103F9800123B6B1255829011F6E024FCF09011F55B
:103FA800E03403F09011F1E0FF123BA3A374FFF09B
:103FB800A3EAF0A3E9F01259E29011F2A3E0FAA300
:103FC800E0AE02FF7A0379FD123B66124FBE12542F
:103FD8005D9011F1E004F0E0C3941E409D9012330F
:103FE800E0FF12592BE4F58475CFE4F5849011F0C5
:053FF800E024FF92AF80
:013FFD0022A1
:03422100901209EF
:10422400123BC6125A1490120AE0FE901209E09052
:10423400120E123BD7E490120DF090120DE0FFC362
:10424400941E504175F0FCEF123B40FE901210F0AA
:10425400FAA3EFF0FB90120BE0FF90120EE0FCA328
:10426400E0FDA9037BFF901220123B6B1256CC9009
:10427400120FE024FCF090120EE03403F090120DC3
:10428400E004F080B5901233E0FF12592BE4F5847A
:0D42940075CFE4F58490120CE024FF92AF8A
:0142A10022FA
:1055C600D296E4FBC295ED25E0FDEC33FC30970462
:1055D600ED4401FDD2950BEBB410E9C296AF05AED2
:0155E60004C0
:0155E70022A1
:0F3BF60075FFDE75FFAD75840F759601758C2018
:103C0500E49012B2F0A3F09012B3E004F0700690C5
:103C150012B2E004F09012B2E0B44EEBA3E0B4208F
:013C2500E6B8
:103C2600759701758A88E4F58475840F75A41175F6
:103C3600A57CF5A675A7E075E12575E344F584F541
:103C46008443E60875DA3175DB3175DC3175DD31B3
:103C560075D983D2DEF584D295C2961255C6E4FC98
:103C6600FDC004C005C006C007AFB0FEEF5403FF99
:103C7600E47810121E0FD003D002D001D000EF4B13
:103C8600FFEE4AFEED49FDEC488F5B8E5A8D59F5E5
:103C960058E55B5401FFE4FEFDFCFBFAF9F8C3129C
:0A3CA6001DFE70037F01227F002243
:10579300010001FF49181510122612280101FFFF0D
:0857A30047B11611122712296B
:10439900900C85E0FBA3E0FAA3E0F9222401F9E4FB
:1043A9003AFAEBF0A3EAF0A3E9F022E0FBA3E47503
:1043B900F001121D66A9F0FA22E0FBA3E475F001F1
:1043C900121D50FA740122E4F0A37407F02204F0DC
:1043D900A37408F0A3742DF02204F0A3740AF0A3C7
:1043E9007453F02204F0A37408F0A37405F02204B6
:1043F900F0A37408F0A37419F0224389204388407C
:04440900758DFE228D
:1045C700E4F58475910575C80475C90875CBFF7541
:1045D700CAFC75CDFF75CCFC53877F759850438E09
:1045E70010124403439802438748D2AC43E740750F
:1045F7008401759850F584438E1053890F12440334
:10460700858D8BD2AC43E740F58453890F438920CE
:10461700758DDF438E10758DE0858D8BD28E7584F9
:084627000143E740E4F58422A1
:10480F00E4900803F0900C83F0A3F07B017A0A790F
:10481F0053900C9A041243AC900C941243ABE49057
:10482F000803F0900C7FF0A3F07A08792D900C9785
:10483F00041243AC900C8E1243AB7A087905900C9E
:10484F008B1243AB900C851243AB7A087919900CFD
:0B485F00911243AB900C881243AB2277
:032A0F00023CB0D6
:103CB000C0E0C0F0C083C082C0D075D000C000C0DA
:0D3CC00001C002C003C004C005C006C0075B
:103CCD0075840030981AC298901292E599F0E0FF31
:103CDD00124DA2901292E0B408069012901243D0A9
:0D3CED0030995D900C7FE07002A3E0604C08
:103CFA00900C9712439C121C17901293F0C299F5DC
:103D0A0099900C7EE004F07006900C7DE004F0902F
:103D1A000C80E024FFF0900C7FE034FFF0900C97C9
:103D2A001243C2900A536B7009E5F065827003EA88
:0A3D3A006583700F900C971243D7B9
:093D44008007C299900C9DE4F087
:103D4D00D007D006D005D004D003D002D001D000CA
:0B3D5D00D0D0D082D083D0F0D0E03274
:032A3F00023D68ED
:103D6800C0E0C0F0C083C082C0D075D000C000C021
:0D3D780001C002C003C004C005C006C007A2
:103D8500758401309811C298AF99EFB40806901266
:103D95009D1243D0124CC830995D900C83E070029F
:043DA500A3E0604CEB
:103DA900900C9A12439C121C1790129FF0C299F51D
:103DB90099900C82E004F07006900C81E004F09078
:103DC9000C84E024FFF0900C83E034FFF0900C9A0F
:103DD9001243C2900C796B7009E5F065827003EAB1
:0A3DE9006583700F900C9A1243E2FC
:0C3DF3008007C299900C9EE4F0758400DB
:103DFF00D007D006D005D004D003D002D001D00018
:0B3E0F00D0D0D082D083D0F0D0E032C1
:104DA200900C85E0FBA3E0FAA3E09012A01243A5C9
:104DB2009012A012439C74019008196B7008E96567
:104DC200827003EA658370069012A01243ED1243CB
:104DD20099EF121C7F9012A0E0F9A3E0FAA3E090F1
:064DE2000C85C91243AC70
:014DE80022A8
:104CC800900C88E0FBA3E0FAA3E09012A31243A59E
:104CD8009012A312439C740190082D6B7008E9652B
:104CE800827003EA658370069012A31243F8900C51
:104CF8008812439CEF121C7F9012A3E0F9A3E0FAFC
:094D0800A3E0900C88C91243AC31
:014D1100227F
:10491800E4F584900C7FE064027004A3E0642660F0
:10492800F2C2AC900C8E1243B4EF121C7F900C8E26
:1049380012439C7401900A536B7008E965827003F6
:10494800EA65837006900C8E1243D7900C80E004C1
:10495800F07006900C7FE004F0900C9DE070040469
:06496800F0D299D2AC224E
:1047B10043E740900C83E064027004A3E064266048
:1047C100F275840153E7BF900C941243B4EF121CAD
:1047D1007F900C9412439C7401900C796B7008E9E2
:1047E10065827003EA65837006900C941243E2902F
:1047F1000C84E004F07006900C83E004F0900C9EB1
:0E480100E0700404F0D29943E740E4F584220D
:1053E600900C8B12439CC003C002C001124399D09B
:1053F60082D083D0E06B7008E965827003EA65832A
:0954060060047F0180027F002296
:10538F00900C9112439CC003C002C001900C881274
:10539F00439CD082D083D0E06B7008E965827003A4
:0C53AF00EA658360047F0180027F002219
:10524400900C8B1243B4121C17FFB408069012B4CE
:105254001243D0900C8B12439C74019008196B700C
:1052640008E965827003EA65837006900C8B12432B
:01527400ED4C
:015275002216
:10527600900C911243B4121C17FFB408069012B694
:105286001243D0900C9112439C740190082D6B70C0
:1052960008E965827003EA65837006900C911243F3
:0152A600F80F
:0152A70022E4
:032A0C00024B4F2B
:104B4F00C0E0C0D075D000C004C005C006C007AF1C
:104B5F0063AE62AD61AC60EC4D4E4F6016EF24FF5B
:104B6F00F563EE34FFF562ED34FFF561EC34FFF5DC
:104B7F0060800C756380756296756198756000D062
:0C4B8F0007D006D005D004D0D0D0E03212
:101718004D6F6E6F00506F6C790020505700416616
:10172800740031006578745F41006578745F420029
:101738006578745F43006578745F44002020203129
:1017480000657874410065787442006578744300D8
:101758006578744400432000432300442000442358
:10176800004520004620004623004720004723006C
:1017780041200041230042200043562025642025B3
:101788007300494E544552504F4C41544500696EC0
:10179800746572706F6C61746500257320782025FC
:1017A8007300256425732E25642078202573002571
:1017B80032642E253032642078202573004C6F6FF8
:1017C80070436F756E746572203D20256400446512
:1017D8006372656D656E74204C2E432E00536574DC
:1017E800204C2E432E203D202564004E6F204A7544
:1017F8006D70004A756D70202B202564004365725A
:101808007461696E7479203D2025642525004A7528
:101818006D7020746F207374616765202564004AB9
:101828006D70546F20253264206966204C433E3029
:10183800005374726F62652041206164647265733D
:1018480073005374616765202564005374726F6276
:101858006520422061646472657373004672656531
:101868000050756C736500537573746E00456E6136
:10187800626C00312F333200312F323400312F3176
:101888003600312F313200332F333200312F3800F8
:10189800312F3600332F313600312F3400312F33BA
:1018A80000332F3800312F3200322F3300332F34DA
:1018B8000077686F6C00332F320032004D756C74FE
:1018C800692054696D65202573002573202A202519
:1018D80032642E25303264207365630054656D7060
:1018E8006F20253364202A20257300436C6F636BB7
:1018F800202A202573005374726F626520256320A7
:10190800616464726573730053746167652025733D
:10191800002535752025357500436F707920546989
:101928006D6520257300436F70696564000053740A
:101938006167652025326420746F20253264004C6D
:10194800434420636F6E74726173743A2564005364
:10195800657474696E6773205361766564005361BA
:1019680076652073657474696E6773005365747463
:10197800696E6773204C6F61646564004C6F6164C5
:101988002073657474696E6773002041424344454F
:10199800464748494A4B4C4D4E4F50515253545567
:1019A800565758595A6162636465666768696A6B15
:1019B8006C6D6E6F707172737475767778797A3032
:1019C8003132333435363738397E21402324255E89
:1019D800262A28292D2B3D7C0101FF4B020104FFFB
:1019E8004DE90108FF56610100FF4B020108FF564F
:1019F800610100FF4E300104FF4DE90108FF566107
:101A08000104FF58C00106FF57EF010BFF580401FE
:101A18000BFF59450011FF2A1C0007FF582D010C28
:101A2800FF5952000EFF582D010CFF59520107FFB4
:101A3800582D0106FF59770106FF59830103FF4F0F
:101A4800F90108FF51DF000BFF4F820108FF59EA37
:101A5800010BFF59F2000BFF4F82010CFF4F4000B2
:101A68000BFF4F820108FF50330014FF2A1C000DA2
:101A7800FF58410000FF59B00000FF591D41424383
:101A880044454647484A4B4C4D4E5000FF1718FFF7
:101A9800171DFF1722FF1726FF172AFF172CFF17FE
:101AA80032FF1738FF173EFF1744FF1749FF174E3D
:101AB800FF1753FF1758FF175DFF1760FF1763FFE6
:101AC8001766FF1769FF176CFF176FFF1772FF176D
:101AD80075FF1778FF177BFF177EFF1864FF1869DB
:101AE800FF186FFF1875FF187BFF1880FF1885FF18
:101AF800188AFF188FFF1894FF1898FF189CFF1872
:101B0800A1FF18A5FF18A9FF18ADFF18B1FF18B558
:091B1800FF18B9FF18BEFF18C246
:1025F10090116474FFF0A37418F0744AA3F0855D20
:1026010082855C83E493FB740193FA7402932290B4
:10261100116474FFF0A37418F0A37405F0E55F244E
:1026210013F582E4355EF583E09011672401FEE441
:1026310033F0CEA3F07B017A11794E2290111174FF
:1026410001F0A37411F0740FA3F090116474FFF002
:10265100A322E55F2404F582E4355EF583E0FDE520
:102661005F2406F582E4355EF583E0FB855F8285B4
:102671005E8322A3F0E55F2414F582E4355EF583E1
:10268100E02401FEE433901167F0CEA3F07B017AE0
:1026910011793D22C9901167F0A3EAF0A3E922FF65
:1026A10090122DE0FBA3E0FAA3E0F922541F901A47
:1026B100EE75F003121EA5E475F003A42583F583DE
:1026C100E493F9222404FFA907E4355EFA7B012291
:1026D100135403FD90110CE075F015A4F58285F0FB
:1026E10083121DA7E5F022FDE4355EFA7464A905A5
:1026F1007B01AD0790126FF022A3F09011DCE07521
:10270100F003A424A0F582E4341AF583E493F922BA
:10271100E55F2405F582E4355EF583E02224F9F9CD
:10272100EA3401FA741CAD0790126FF0221258E1DD
:10273100E4901167F0A3EF22FFE4355EFE7C00EF29
:102741002526FFEC3EFAA9077B01E0FD90126F22DE
:102751009011117401F0A322F99001F9021C30E0EB
:10276100FBA3E475F001121D66A9F0FA021C1774AF
:1027710001F0A37411F0A37460F022A3A3E0FEA3FF
:10278100E0FF541FD39410E49400222FF9EA35F0AE
:10279100FAE92402F9E43AFAEB2275F005A4241EC1
:1027A100F582E43411F5832275F005A4241CF58229
:1027B100E43411F5832275F005A4241DF582E43477
:1027C10011F58322A3A3EF54E04410FFEEF0A3EF31
:1027D100F0229012637401F0A37411F0A3744E22DD
:1027E100CFF0A3EFF0900C81E0FFA3E0229012C0A4
:1027F100E4F0A37407F022FFE4355EFAA907901212
:102801002DEB22A3A3E0FCA3E0FD227401F0A3744D
:1028110011F0A37415F022855D82855C83740693A3
:10282100F8E622AD0790126FF022A3F0900C79E048
:0E283100FFA3E022A3F0900C7BE0FFA3E022C7
:10562700E490110FF090111BF0901119F0901110E8
:0E563700F090113BF090115FF090113CF022CA
:065A2600E4901114F022CF
:10455D009012B8EEF0A3EFF0AF051DEF605B901277
:10456D00B8E0FEA3E0F5828E83A3A3122605F99091
:10457D001114E0FF12279BEB122699F09012B8E070
:10458D00FAA3E0FBF5828A83E493FEEF1227A9EEEE
:10459D00F08B828A83740193FF901114E01227B778
:1045AD00EFF0901114E004F09012B9E02405F090B2
:0A45BD0012B8E03400F00245652258
:104B9B00901114E0FF60449011111226A4121C17FF
:104BAB00C39F4004E4121C7F9011111226A4121C07
:104BBB0017FE1227A9E0FFEE1227B7E0FD12596B83
:104BCB009011111226A4121C1712279BE0F9A3E0D7
:0C4BDB00FAA3E0901116C9122699F022EE
:10567D009011111226A47401121C5D121C17FF90BB
:0B568D001114E0B50704E4121C7F229A
:012A1B002298
:0F59000090111674FFF0A3742AF0A3741BF02209
:104C7D009012BAEEF0A3EFF0AF05EF3395E0FEE042
:104C8D002FF09012BAE03EF0E0FEA3E0FFBEFF0C65
:104C9D00BFFF09E49012BAF0A3F08016EFB503122E
:104CAD00EEB5020EEB24FFFEEA34FF9012BAF0A32C
:0B4CBD00CEF09012BAE0FEA3E0FF2250
:1029E40090126BEB122699F090126B1226A4121C13
:1029F40017FF7E0090126FE0FB7A00124C7D90125C
:082A04006B1226A4EF021C7FF7
:104B0200AC07300021E55F1226C5AD0490126F7428
:104B12000FF01229E4E55F2404122715640A702AB3
:104B2200E55F2406801BE55F24051226C7AF0474E7
:104B32000F1227271229E4122711B40A0DE55F2468
:0D4B420007F582E4355EF583E4F00253369A
:10440D0090122AEB122699F090122A1226A4121C51
:10441D0017B40A08901230E064016054901231E034
:10442D00FF901230E08FF0A41226A0EF121C5D1247
:10443D001C17D3648094E34004749C80281226A139
:10444D00121C17C364809480502690122A1226A441
:10445D00121C17700B901231E01226A0EF021C5D9A
:10446D001226A17464121C5D901230E0FF124B02F3
:01447D00221C
:104DE9009012C8EFF0E55F30000F1226C5C003C06E
:104DF90002C001E55F2406800F24051226C7C003FF
:104E0900C002C001E55F24071227F8122699F09025
:104E190012C8E0901230F0A37401F0D001D002D092
:074E29000312440D02533691
:10566100E55F300004240880022409FDA905122603
:0C567100CA74051228241229E4025336E2
:104E30009012C9EFF0E55F30000F1226C5C003C025
:104E400002C001E55F2406800F24051226C7C003B7
:104E5000C002C001E55F24071227F8122699F090DE
:104E600012C9E0901230F0A3740AF0D001D002D041
:074E70000312440D0253364A
:1058C0007B007A00792674041228241229E40253FA
:0158D00036A1
:1057EF009012CAEFF0E55F240A1227397466F0129F
:0557FF0029E40253360D
:105804009012CBEFF0E55F240E1227397415F012D5
:0558140029E4025336F7
:0D594500E55F24121226E81229E402533611
:012A1C002297
:10582D00E55F2414FDE4355EFA74181226EF122993
:04583D00E4025336F8
:0D595200E55F24131226E81229E402533603
:0C5977001225FF12271E1229E4025336ED
:0C5983001225FF12271E1229E4025336E1
:104FF900AD0712266DA3A37E00A3E05407FF7B052E
:105009007A00124C7DEF5407FF12266DA3A3C083CB
:10501900C082E0FCA3E054F8FDECFEED4FFFD08226
:0A502900D083EEF0A3EFF00253363F
:1051DF00AD0712266DA3A3E05407FEA3E0FF7BE704
:1051EF007A03124C7DEE5407FE12266DA3A3C083E3
:1051FF00C082E054F84EFED082D083EEF0A3EFF0E1
:03520F0002533611
:104F8200AD0712266DE0C41354077E005403FF7B65
:104F9200047A00124C7DEF5403C43354E0FE12260F
:104FA2006DC083C082E0549FFCA3E0FDEC4EFFED98
:0C4FB200D082D083CFF0A3EFF002533682
:1037FA009012BCEFF0A3EDF08FF0A4F012266DA3A7
:10380A00A3C083C082E0FCA3E0FD9012BDE0F9FBF7
:10381A003395E0FAEDAE047803CEC313CE13D8F98C
:10382A00FFEE541FFE7C00ED5407FDEF2BFFEE3A2E
:10383A00541FFEEF7803C333CE33CED8F9FFEC4ED4
:10384A00FEED4FFFD082D083EEF0A3EFF0E96401E2
:10385A00702C12266D122804AE047803CEC313CE40
:10386A0013D8F9FFEE541FFEEF64014E70101226B2
:10387A006DA3A3ED54074410FFE4F0A3EFF0122662
:10388A006D122804AE047803CEC313CE13D8F9FF01
:10389A00EE541FFED3EF94B8EE940B40339012BC53
:1038AA00E0D364809480401112266DA3A3ED5407DF
:1038BA00FFEF44C0FF745D801312266DA3A3C0837B
:1038CA00C082A3E05407FFD082D083E4F0A3EFF0D4
:0138DA0022CB
:0859EA007D641237FA02533606
:0859F2007D011237FA02533661
:104F4000AD0712266DA3A3E0131313541F7E005464
:104F50001FFF7B117A00124C7DEF541F3333335403
:104F6000F8FE12266DA3A3C083C082E05407FCA301
:104F7000E0FDEC4EFFEDD082D083CFF0A3EFF00246
:024F80005336A6
:10503300AD0712266DA3A37E00A3E0541FFF7B11CF
:105043007A00124C7DEF541FFF12266DA3A3C08379
:10505300C082E0FCA3E054E0FDECFEED4FFFD08204
:0A506300D083EEF0A3EFF002533605
:105841007B017A127934AD0790126F7408F0122936
:04585100E402598F85
:0B59B000201E05E4FF1252D8D21E2278
:0E591D00201B081254F27F0412496ED21B2286
:08283F009011D9EDF0A3EBF0BC
:102847009011DCE0D394044009A31227F1E490111E
:10285700DCF01227517411F0745F1226497417F0D7
:10286700A37481F07C003000047D0180027D02901A
:102877001167ECF0A3EDF0EF7BFF60067A17798A1A
:1028870080047A177996901169EBF0A3EAF0E912C0
:10289700268C121F8E9011D9E0FFD3940A403F1265
:1028A700264B7417F0A374A2F0EF75F003A42482EB
:1028B700F582E4341AF583E493F912260812269573
:1028C7001226FB12260890116AC9F0A3EAF0E91252
:1028D7002634121F8E7E197FEF7D020229DE9011AA
:0728E700DBE070030229A7EA
:1028EE009011D9E075F064A4FFA3E07C002FFEECFC
:1028FE0035F09011DFF0A3CEF09011DFE0FAA3E0F7
:10290E00FB7D78FFAE02121CC5A3EFF0E075F078E8
:10291E00A4FFC3EB9FFFEA95F0FE7C007D0A121C1C
:10292E00C5A3EF12264A7417F0A374AAF09011E112
:10293E00E0FEFD901167E4F0A3EDF0EF75F003A457
:10294E0024BEF582E4341AF583E493F91226089036
:10295E001169C9122699F0EE75F078A4FFC3901193
:10296E00E0E09FFD9011DFE095F0FC9011E2E07544
:10297E00F00AA4FFC3ED9FFEEC95F090116CF0CE23
:10298E001226FA12260890116EC9122699122635B1
:07299E00121F8E7E197FF964
:1029A500803512264B7417F0A374B7F09011D9E057
:1029B500FF122731F09011DAE0FF901169E4F0EF92
:1029C5001226FA12260890116BC91226991226357D
:0F29D500121F8E7E197FE07D0312455D02586848
:1058E1007493B55D087457B55C03AF1722AF1822E6
:104322001227517411F0A37419F012272E12264A83
:104332007417F0A374C512268D121F8E12266DE01B
:10434200FEA3E07807CEC313CE13D8F9540314604A
:104352000E14601C2402703CE490114EF080351261
:10436200264B7417F0A374D6122635121F8E8024A2
:1043720012264B7417F0A374E5F0E55F241212279E
:1043820015FF122731122635121F8E7E1A7F177DD6
:074392000112455D025868AD
:104119001227517411F0A3741BF07E1A7F1C7D06BF
:1041290012455D12266DE0C313540314601914601F
:104139002A14603A2403705C12264B7417F0A37496
:10414900F312268D02419A12264B7417F074FB1252
:104159002674121F8E12261002419A12264B7418C9
:10416900F07416122674121F8E122610802312273D
:104179002E12264A7417F0A374C512268D121F8EAB
:1041890012264B7418F0A37427F0E55F2414122645
:0741990022121F8E0258687C
:10553B0012263D7418F0A3743912268D121F8E1289
:10554B0025F112275912262A121F8E7E1A7F3A7DB9
:04555B000102455DA7
:10540F0012263D7418F0A3745312268D121F8E129C
:10541F0025F112275912262A121F8E7E1A7F3F7DE1
:07542F000112455D025868FF
:102C150012264B7418F0A374C4F012266DE0C41389
:102C25005403901AE21226B212260812269512268D
:102C35008D121F8E12266DE01313135403147003A7
:102C4500022CFC147003022D5E24026003022D9EEB
:102C550012266DA3A3E0FEA3E07803CEC313CE1323
:102C6500D8F9FFEE541FFEAB07FA7C007D64121DF8
:102C75001A9012BEEEF0A3EFF09012BEE0FEA3E0B4
:102C8500FF7C007D64121CB3C3EB9FFFEA9EFE90A0
:102C950012BEE07002A3E07007EF4E7003FE7F01E5
:102CA50012264B7418F0A374D2F012266DA3A3A3B9
:102CB500E05407901AAF1226B2122608122695F094
:102CC5009012BEE0FDA3E090116ACDF0A3EDF0A354
:102CD500EEF0A3EF122635121F8EE5339011116029
:102CE5000A12280C7E1A7F44022D4D1227707E1A77
:102CF5007F4E7D03022D9B12266D12277C40061206
:102D0500266D1227C512264B7418F0A374E4F01231
:102D1500266D122804EC5407FEED2401FFE43E1253
:102D25002732F0EC1313131226AD12260890116901
:102D3500C9122699122635121F8EE533901111609E
:102D45000C12280C7E1A7F497D01022D9B122770DB
:102D55007E1A7F5D7D02022D9B12266D12277C4017
:102D65000612266D1227C512264B7418F0A374F3AC
:102D7500F012266DA3A3A3E01226AD122608122693
:102D850095122635121F8E30100F122751122774F7
:0C2D95007E1A7F677D0212455D025868BF
:10408D0012263D7418F0A374FEF07493B55D097497
:10409D0057B55C047F4180027F42901167EF122675
:1040AD008D121F8E1225FF122759FFC3941850161B
:1040BD0012264B7418F0A3744AF0EF2401FEE4337A
:1040CD00A3F0A3CE80371225FF122759D3941C409D
:1040DD00089001F97418121C9112264B7419F07482
:1040ED00101225FD12275975F003A4245BF582E407
:1040FD00341AF583E493F912260812269512263503
:0C410D00121F8E7E1A7F3A7D0102455D74
:1039B700900C7DE0FEA3E0FF901103E0B50641A364
:1039C700E0B5073C900C81E0FEA3E0FF901105E015
:1039D700B5062DA3E0B50728900C79E0FEA3E0FF1C
:1039E700901107E0B50619A3E0B50714900C7BE02A
:1039F700FEA3E0FF901109E06E7003A3E06F607211
:103A070012264B7419F0741912282BCF122732F093
:103A1700900C7DE0FFA3E0901169CFF0A3EF122691
:103A27008D121F8E12264B7419F0741912283590B7
:103A370011671227E1901169CFF0A3EF1226351213
:103A47001F8E900C7DE0FFA3E09011031227E190F9
:103A57001105CFF0EF12282B901107CFF0EF1228A6
:103A670035901109CFF0A3EFF01227D312268D124C
:023A77005145B7
:013A7900222A
:105855001227517411F0A3741AF07E1A7F717D011D
:0358650002455D9C
:103FFE001225FFF9740693F8E61226D9131312262A
:10400E00D113131354036D7001E47020855D828506
:10401E005C83122606F9740693F8E61226D9C412AA
:0F402E0026D1C41354036D7001E460037F002298
:10403D0012281875F015A4FF1226059012471227A5
:10404D008C1226991225FEF990110CE075F015A42D
:10405D00FFE990124A12278C122699F0A37402F0F0
:10406D0090124DE0FF14F0EF601390124A1227608A
:0D407D00FF9012471227606F60E67F00225F
:03408A007F012291
:1038DB001227517411F0A3740DF090110EE01460C7
:1038EB006214607814700302398D2403600302396B
:1038FB00B6123FFEEF7BFF60067A19792E80047AB1
:10390B00197935EB12269612264A7419F0A37421F5
:10391B0012268D121F8E12264B7419F0A37436F0DB
:10392B0090110CE02401FEE433901167F0A3CEF06C
:10393B0012281890116912262D121F8E7E1A7F7174
:10394B000239B112264B7419F0A37447F09012345C
:10395B00122681121F8E7E1A7F76804A9011647414
:10396B00FF301E0AF0A37419F0A374578008F0A35C
:10397B007419F0A3746612268D121F8E7E1A7F7B2C
:10398B00802490116474FF301B0AF0A37419F0A308
:10399B0074748008F0A37419F0A3748412268D122A
:0C39AB001F8E7E1A7F807D0112455D2278
:10360A00E55F2408122715D3940440031227EEE538
:10361A005F2409122715D3940440031227EE125A85
:10362A0026E490114EF090113DF02006030237096E
:10363A003002061238DB02370C30001D12266DA349
:10364A00E05401FFC007122653E0FEA3E07802CE41
:10365A00C313CE13D8F90236BD30013212266DE0FB
:10366A00C313A3E0135401FFC007122711FDE55F3E
:10367A002407122664E0FEA3E07803CEC313CE1318
:10368A00D8F954019011DBF0E55F2409802F30044A
:10369A003A200005200102D20012266DA3E054014F
:1036AA00FFC007122653E0FEA3E07802CEC313CE72
:1036BA0013D8F954019011DBF0E55F24081227159D
:1036CA009011DCF0D00712283F80373007051243EB
:1036DA0022802F3008051241198027300C05125517
:1036EA003B801F300D0512540F8017E533700330ED
:1036FA001005122C15800B30030812408D8003121E
:0E370A0058551227D312268D125145024B9BA3
:03000000020C00EF
:03000300022A03CB
:03000B00022A06C0
:03001300022A09B5
:03001B00022A0CAA
:03002300022A0F9F
:03002B00022A1294
:03003300022A1589
:03003B00022A187E
:03004300022A1B73
:03004B00022A1E68
:03005300022A215D
:03005B00022A2452
:03006300022A2747
:03006B00022A2A3C
:03007300022A2D31
:03007B00022A3026
:03008300022A331B
:03008B00022A3610
:03009300022A3905
:03009B00022A3CFA
:0300A300022A3FEF
:100C0000787FE4F6D8FD9000007F007E20E4F0A31A
:0A0C1000DFFCDEFA758167020C5567
:100C1A00020C9AE493A3F8E493A34003F68001F24A
:100C2A0008DFF48029E493A3F85407240CC8C333DB
:100C3A00C4540F4420C8834004F456800146F6DFAA
:100C4A00E4800B01020408102040809053BBE47E2C
:100C5A00019360BCA3FF543F30E509541FFEE4939F
:100C6A00A360010ECF54C025E060A840B8E493A366
:100C7A00FAE493A3F8E493A3C8C582C8CAC583CA91
:100C8A00F0A3C8C582C8CAC583CADFE9DEE780BE49
:0153E50000C7
:101B2100E709F608DFFA8046E709F208DFFA803EA6
:101B310088828C83E709F0A3DFFA8032E309F60893
:101B4100DFFA8078E309F208DFFA807088828C83FB
:101B5100E309F0A3DFFA806489828A83E0A3F608AF
:101B6100DFFA805889828A83E0A3F208DFFA804C89
:101B710080D280FA80C680D4806980F28033801060
:101B810080A680EA809A80A880DA80E280CA8033C9
:101B910089828A83ECFAE493A3C8C582C8CCC58341
:101BA100CCF0A3C8C582C8CCC583CCDFE9DEE78011
:101BB1000D89828A83E493A3F608DFF9ECFAA9F090
:101BC100EDFB2289828A83ECFAE0A3C8C582C8CCE6
:101BD100C583CCF0A3C8C582C8CCC583CCDFEADEFF
:101BE100E880DB89828A83E493A3F208DFF980CC61
:101BF10088F0EF60010E4E60C388F0ED2402B4045A
:101C01000050B9F582EB2402B4040050AF23234500
:061C11008223901B717399
:101C1700BB010689828A83E0225002E722BBFE02CB
:091C2700E32289828A83E49322FE
:101C3000BB010CE58229F582E5833AF583E0225069
:101C400006E92582F8E622BBFE06E92582F8E222B3
:0D1C5000E58229F582E5833AF583E49322CD
:101C5D00BB010989828A83F8E028F022500327F717
:101C6D0022BBFE05F8E328F3228A838982F8E493E8
:021C7D0028221B
:101C7F00BB010689828A83F0225002F722BBFE0144
:021C8F00F3223E
:101C9100F8BB010DE58229F582E5833AF583E8F089
:101CA100225006E92582C8F622BBFE05E92582C835
:021CB100F2221D
:101CB300EF8DF0A4A8F0CF8CF0A428CE8DF0A42E45
:021CC300FE22FF
:101CC500BC000BBE0029EF8DF084FFADF022E4CC03
:101CD500F875F008EF2FFFEE33FEEC33FCEE9DECCC
:101CE500984005FCEE9DFE0FD5F0E9E4CEFD22ED12
:101CF500F8F5F0EE8420D21CFEADF075F008EF2F5C
:101D0500FFED33FD4007985006D5F0F222C398FD4C
:051D15000FD5F0EA22E9
:101D1A00C2D5EC30E709B2D5E4C39DFDE49CFCEEE4
:101D2A0030E715B2D5E4C39FFFE49EFE121CC5C37B
:101D3A00E49DFDE49CFC8003121CC530D507C3E476
:061D4A009FFFE49EFE2253
:101D5000C5F0F8A3E028F0C5F0F8E582158270021E
:061D60001583E038F022BB
:101D6600A3F8E0C5F025F0F0E58215827002158330
:061D7600E0C838F0E8228D
:101D7C00BB010A89828A83E0F5F0A3E02250068732
:101D8C00F009E71922BBFE07E3F5F009E3192289F4
:0B1D9C00828A83E493F5F07401932227
:101DA700BB0110E58229F582E5833AF583E0F5F07A
:101DB700A3E0225009E92582F886F008E622BBFE57
:101DC7000AE92582F8E2F5F008E222E5832AF5839D
:081DD700E993F5F0A3E9932262
:101DDF00BB010A89828A83F0E5F0A3F0225006F74F
:0F1DEF0009A7F01922BBFE06F3E5F009F319224C
:101DFE00EB9FF5F0EA9E42F0E99D42F0E89C45F03B
:011E0E0022B1
:101E0F00E8600FEFC333FFEE33FEED33FDEC33FC31
:031E1F00D8F122D5
:101E22007401FF3395E0FEFDFCA3A3A3E0CF2FF0E6
:101E3200E582158270021583E0CE3EF0E5821582BE
:101E420070021583E0CD3DF0E582158270021583A4
:051E5200E0CC3CF02291
:0C1E5700ECF0A3EDF0A3EEF0A3EFF022FE
:101E6300A8828583F0D083D082121E7A121E7A1242
:101E73001E7A121E7AE473E493A3C583C5F0C58367
:101E8300C8C582C8F0A3C583C5F0C583C8C582C8C9
:011E9300222C
:101E9400F5F0C582A4C582C5F0C583A42583F58366
:011EA400221B
:0C1EA500A42582F582E5F03583F5832248
:101EB100D083D082F8E4937012740193700DA3A3C0
:101EC10093F8740193F5828883E4737402936860D4
:061ED100EFA3A3A380DFD4
:061ED7008A838982E47396
:101F2900E51B2464F582E43411F583E0051B229056
:101F39001161301803901164E475F001121F090250
:101F49001C172011E97F2ED2118018EF540F24900D
:101F5900D43440D4FF30150BEF24BFB41A0050031A
:101F69002461FFE51C6002151C051FE51F700205B1
:101F79001E30180E901161E475F001121F09EF026D
:101F89001C7F0254367403D2188003E4C218F51B6F
:101F9900901161121F20E4F51CF51EF51FE51C6068
:101FA900077F20121F6C80F5751DFFC212C211C276
:101FB90013C214C216C217C219121F38FF700D308E
:101FC90018057F00121F7DAF1FAE1E22B4255FC208
:101FD900D5C215121F38FF24D0B40A00501A75F063
:101FE9000A781C30D50508B6FF0106C6A426F620D6
:101FF900D5047002D21480D924CFB41A00EF50044A
:10200900C2E5D21502217ED21280C6D21180C0D279
:102019001380BCD2D580BAD21680B47F20121F6C2F
:102029002013077401B51C0040F1121F29FF121F6C
:102039006C021FA6D219D2178095121F29FB121FF5
:1020490029FA121F29F94A4B7006794F7A227BFF28
:1020590020132EE51C602A7E008E82758300121CD7
:102069003060060EEE651D70F0C2D5EBC0E0EAC027
:10207900E0E9C0E0EE1221C5D0E0F9D0E0FAD0E005
:10208900FB121C17FF60AAEBC0E0EAC0E0E9C0E060
:10209900121F6CD0E02401F9D0E03400FAD0E0FB43
:1020A900E51D0460DCD51DD980877BFF7A2179C1C4
:1020B900D213809C791080027908C217C21980084E
:1020C900D2D5790A8004790AC2D5E51D047002F5D2
:1020D9001DE4FAFDFEFF121F29FC7B0820121312D2
:1020E9001F29FD7B1030110A121F29FE121F29FF1B
:1020F9007B20EC3382D592D55013C3E43011069F6F
:10210900FFE49EFEE42012039DFDE49CFCE4CBF871
:10211900C212EC700CCFCECDCCE824F8F870F38065
:1021290017C3EF33FFEE33FEED33FDEC33FCEB3336
:10213900FB994002FB0FD8E9EB301205F8D0E0C457
:1021490048B212C0E00AEC4D4E4F78207B0070C2B5
:10215900EAB51D0040BCC0E01221C7D0F0D0E02094
:102169001204C4C0E0C4B212C0F0121F55D0F0D599
:10217900F0EB021FA6121EB120435320BD582014B4
:102189004C20104220C14F20C94420C9492029436D
:0821990020CF5520B34620B30E
:1021A1004520B347226F5020182D201C2E203F2B95
:1021B100202023203D2022582A1FD8480000203704
:1021C1003F3F3F00790AA2D5201414301609B910F7
:1021D100020404B9080104A2D52017025001042009
:1021E10013689213B51C005034C0E07F20301419DD
:1021F1007F30A21372177216500F12221EC213C221
:1022010017C216C2197F30800F301603E9C0E012E1
:102211001F6C301603D0E0F9D0E0B51CCC30161796
:102221007F30B9100C121F6C7F583015077F7880F2
:1022310003B90803121F6C3013057F2D021F6C7F39
:10224100202019F87F2B2017F322921380CF286EBC
:10225100756C6C2900D212121F293012F8C2127843
:102261001C30D50108F6021FD82D50434958121FC2
:10227100292403B405004001E490226A93121F5DF2
:0D228100743A121F5DD214751C040220BDBA
:101EDD00EF4E6012EF60010EEDBB010B89828A831C
:101EED00F0A3DFFCDEFA2289F05007F709DFFCA929
:0C1EFD00F022BBFEFCF309DFFCA9F02280
:101F0900F8E0FBA3A3E0F925F0F0E5821582700261
:071F19001583E0FA38F02205
:091F2000EBF0A3EAF0A3E9F022C2
:10543600EFB40A07740D125441740A309811A899F2
:10544600B8130CC2983098FDA899C298B811F630D6
:0754560099FDC299F59922AE
:00000001FF
